:020000040000FA
:0600000001EF1EF01200EA
:0608000001EF1EF01200E2
:06080800E1EF04F0120014
:060818001CEF04F01200C9
:06082A0001002E3C00005D
:08083000EC0200000A000000C8
:08083800D8CFE4FFE0CFE4FF9C
:10084000E46EDACFE4FFE2CFDAFFE9CFE4FFEACFEC
:10085000E4FFF3CFE4FFF4CFE4FFE6529EA270D0B2
:100860009E920001000ED880E655000EE75534E256
:100870000201EC2B000EED230001E6510201EC5DBC
:100880000001E7510201ED5927E3EC6BED6B030E1C
:100890000001EA5D1FE2E851EA6AC80FE96E020E44
:1008A000EA2280CFEFFFE851EA6ACB0FE96E020E31
:1008B000EA2281CFEFFFE851EA6ACE0FE96E020E1D
:1008C000EA2282CFEFFFE82B030EE85D01E3E86B3D
:1008D000EA2B02D0E66BE76B0001000ED880EB55E7
:1008E000000EEC551FE2F05100081CE20201EE2B55
:1008F000000EEF230001EB510201EE5D0001EC510F
:100900000201EF590FE3EE6BEF6B030E0001EF5D99
:1009100007E2ED2B030EED5D01E3ED6BEF2B02D053
:10092000EB6BEC6B0001F05100080AE2F16BF15146
:10093000040DF328C26E9E9C9F9C9D8CC280C28237
:100940009EAC2ED09E9CC450266E26C027F0266AF0
:10095000C35000012610246E27C025F00001F1517C
:10096000060DF3CF22F0F4CF23F0800E2226020EE4
:100970002322ED51020D2250F324E96E2350F4207E
:10098000EA6E24C0EEFF25C0EDFFF12BF051F15DC2
:1009900002E39D9C05D0F151040DF328C26EC28282
:1009A000E552E5CFF4FFE5CFF3FFE5CFEAFFE5CF72
:1009B000E9FFE5CFDAFFE550E5CFE0FFE5CFD8FF6F
:1009C0001000DACFE4FFE2CFDAFFE652E552E5CFDE
:1009D000DAFF1100D9CFE6FFE1CFD9FF020EE12601
:1009E000896A92680F0EC16E070EB46E8A6A9368A8
:1009F0008B6A9468FC0E8B16941694848250040BB8
:100A000001E0010E0001606FE26BE36BEE6BED6BDA
:100A1000EF6BE96BE86BEA6BE66BE76BEB6BEC6B30
:100A2000CA82CA80CA9CCA9ACA88CA96FA0ECB6E73
:100A3000DF6ADFCF14F00C0EE76E1418E8AE02D0B8
:100A4000E73402D0E750145C36E2010EDB6ADBCFFC
:100A500014F0030EE76E1418E8AE02D0E73402D0AB
:100A6000E750145C26E2DFCF14F0156A14BE156857
:100A7000060E1502F3CF15F01402F3CF14F0F45064
:100A80001526800E1426020E1522010EDBCF16F05D
:100A9000176A16BE1768D8901636173614501624E3
:100AA000E96E15501720EA6EEE6AED6A010EDB2A38
:100AB000CED7DF2ABED7D08ECA949D829F92F28E67
:100AC000F28CCA84020EE15C02E2E16AE552E16E58
:100AD000E552E7CFD9FF1200D9CFE6FFE1CFD9FF2A
:100AE000080EE126010EDF6EDB6A020EDB6A030EE2
:100AF000DB6A86EC0FF0060E0001FC5D03E36D502F
:100B0000020B01E03AD10001EA51000843E2020180
:100B1000D25140E10001E951EA6ACE0FE96E020EBE
:100B2000EA22EF50E66EE66AE951EA6ACB0FE96E17
:100B3000020EEA22EF50E66EE66AE951EA6AC80F51
:100B4000E96E020EEA22EF50E66EE66A610E146E5E
:100B50003B0E156E166A14C0E6FF15C0E6FF16C000
:100B6000E6FFA10EE66E000EE66E28EC1CF0176E96
:100B70000B0EE15E17500001E92B030EE95D01E168
:100B8000E96BEA07A10EE66E000EE66E97EC16F032
:100B9000E552E5520001EF51000801E39CD002014B
:100BA000D25101E098D0060EDB6ADBCFE9FFEA6A9A
:100BB000E9BEEA68A10EE926000EEA22410EEF6EB8
:100BC000060EDB2A070EDB6A0001F051F36E070EFA
:100BD000DBCFF4FFF350F45C4BE2070EDBCF14F0F5
:100BE000156A14BE1568060E1502F3CF15F014022F
:100BF000F3CF14F0F4501526800E1426020E1522A1
:100C0000EE51020D1450F324E96E1550F420EA6EF3
:100C1000EECFE6FFEFCFE6FF5B0E166E3B0E176ED4
:100C2000186A16C0E6FF17C0E6FF18C0E6FF060EFA
:100C3000DBCF19F01A6A19BE1A68A10E1926000E28
:100C40001A2219C0E6FF1AC0E6FF28EC1CF01B6E42
:100C5000070EE15E1B50050E146E060EDBCFE7FF9C
:100C60001450E726060EE7CFDBFF070EDB2AACD7D2
:100C7000060EDBCFE9FFEA6AE9BEEA68A10EE926C3
:100C8000000EEA220A0EEF6E060EDB2ADBCFE9FF2A
:100C9000EA6AE9BEEA68A10EE926000EEA220D0E14
:100CA000EF6E060EDB2ADBCFE9FFEA6AE9BEEA68EF
:100CB000A10EE926000EEA22EF6AEE2B030EEE5D8E
:100CC00001E1EE6BEF07A10EE66E000EE66E97EC0B
:100CD00016F0E552E552400EE66E610EE66E000E2D
:100CE000E66E57EC16F0E552E552E552E76E010E5E
:100CF000E7CFDBFF0001E16BDBCF14F0000EE76E06
:100D00001418E8AE02D0143403D0E750D88014543D
:100D100005E2010EDBCFE6FF3AD8E552D950040FC9
:100D2000E66E000EDA20E66EA0D8E552E552000924
:100D300024E0040EDBCFE6FF11D9E552000E0001DE
:100D4000E76EE119E8AE02D0E13503D0E750D88074
:100D5000E15513E20201D25110E1E1C0A1F000011E
:100D60000D0EA26F0A0EA36FA46BA10EE66E000E0D
:100D7000E66E97EC16F0E552E552080EE15C02E2F1
:100D8000E16AE552E16EE552E7CFD9FF1200D9CF13
:100D9000E6FFE1CFD9FFE652DF6AFE0EDB50DF5CF3
:100DA0005FE20201F35123E10D0E146EDF50EA6A97
:100DB000610FE96E000EEA22EF50145C0BE00A0EA0
:100DC000156EDF50EA6A610FE96E000EEA22EF50FD
:100DD000155C0DE1010EF36F0001E251EA6A000FAC
:100DE000E96E020EEA220D0EEF6EE22B28D0DF50E4
:100DF000EA6A610FE96E000EEA22EF500D081FE06B
:100E0000DF50EA6A610FE96E000EEA22EF500A082D
:100E100016E0DF50EA6A610FE96E000EEA22EF5039
:100E2000E66E0001E251EA6A000FE96E020EEA2264
:100E3000E552E750EF6E0201F36B0001E22B000177
:100E4000E251146E156A800E141802E1000E151896
:100E500001E1E26BE351E25D01E102D0DF2A9DD7BF
:100E6000E552E552E7CFD9FF1200D9CFE6FFE1CF37
:100E7000D9FF020EE126010EE3C0DBFFDB500001CB
:100E8000E25D0AE1FD0EDBCFE9FFFE0EDBCFEAFFFC
:100E9000EF6A616B000E56D0DF6ADF50146E156A80
:100EA000D890155004E6800E145C000E155840E2F0
:100EB000010EDB50EA6A000FE96E020EEA22EF50E3
:100EC000E66EDF50EA6A610FE96E000EEA22E55233
:100ED000E750EF6E010EDB2ADB50146E156A800EB0
:100EE000141802E1000E151802E1010EDB6A0D0E66
:100EF000146EDF50EA6A610FE96E000EEA22EF50CD
:100F0000145C0FE1DF28E66EFD0EDBCFE9FFFE0E7D
:100F1000DBCFEAFFE552E750EF6E010EDBCFE3F0E7
:100F200011D0010EDB50E25D01E102D0DF2AB5D71E
:100F3000FD0EDBCFE9FFFE0EDBCFEAFFEF6A616B50
:100F4000000E00D0146E020EE15C02E2E16AE5528E
:100F5000E16E1450E552E7CFD9FF1200D9CFE6FF7A
:100F6000E1CFD9FFFE0EDB040BE0FE0EDB500208E2
:100F70000BE22C0E0001625D07E02C0E635D04E0C5
:100F800000012C0EE16F7CD0FE0EDB04EA6A610FDB
:100F9000E96E000EEA22EF500D0804E00001210E78
:100FA000E16F6ED0000161514D0A5BE01D0A46E021
:100FB000040A35E0150A31E0170A2DE01F0A29E07E
:100FC000060A25E00C0A14E0110A03E03F0EE16F67
:100FD00057D06251580A07E0740A03E03F0EE16FF0
:100FE0004FD052D804D05CEC0DF001D000D048D0E6
:100FF0006251580A07E0740A03E03F0EE16F40D0E7
:10100000B1D804D05DEC0DF001D000D039D039D981
:1010100037D096D935D0BED933D0C8D931D0625166
:10102000580A07E0740A03E03F0EE16F29D02ED87A
:1010300004D05BEC0DF001D000D022D06251440A04
:101040000CE00B0A07E0060A03E03F0EE16F18D040
:10105000C1DB06D09AEC0CF003D0FBDA01D000D053
:101060000FD06251570A07E0050A03E03F0EE16F17
:1010700007D084DA03D02CDA01D000D001D000D020
:10108000E552E7CFD9FF1200EAEF04F0D9CFE6FF2F
:10109000E1CFD9FF020EE126010EDF6EDB6A030EFF
:1010A000E66ED9CFE6FFDACFE6FF5FEC0DF0E55252
:1010B000E552E55207C0E4F008C0E5F0010EE66E27
:1010C000D9CFE6FFDACFE6FF5FEC0DF0E552E5524F
:1010D000E552010E07C0DBFF0001E15101E038D00D
:1010E000DF50EA6A610FE96E000EEA22EF500D0848
:1010F00005E0E15103E1230EE16F2AD0E15128E13F
:10110000010EDB5013E1E451E51103E1E66BE76BFF
:101110000CD00A0EE45D000EE55903E20A0EE46FFE
:10112000E56BE4C0E6F0E5C0E7F012D0E451E5116C
:1011300003E1EB6BEC6B0CD00A0EE45D000EE5599D
:1011400003E20A0EE46FE56BE4C0EBF0E5C0ECF0FF
:10115000020EE15C02E2E16AE552E16EE552E7CFA0
:10116000D9FF1200D9CFE6FFE1CFD9FF050EE12666
:10117000010EF36E040EF3CFDBFF010EE66ED950C5
:10118000040FE66E000EDA20E66E5FEC0DF0E5521D
:10119000E552E5520750DF6E010EE66ED950040F9E
:1011A000E66E000EDA20E66E5FEC0DF0E552E552D9
:1011B000E552010E07C0DBFFE66ED950040FE66E64
:1011C000000EDA20E66E5FEC0DF0E552E552E552D6
:1011D000020E07C0DBFF010EE66ED950040FE66E6B
:1011E000000EDA20E66E5FEC0DF0E552E552E552B6
:1011F000030E07C0DBFF0001E15101E038D0040E0F
:10120000DB50EA6A610FE96E000EEA22EF500D082A
:1012100005E0E15103E1230EE16F29D0DF50926E2A
:10122000010EDB50936E020EDB50946E030EDB500A
:101230000C0805E20C0EF36E030EF3CFDBFF030E7A
:10124000DB5005E10F0EC16EC290F06B10D0F06B59
:10125000C26A030EDBCFE6FF0F0EE552D880E754DB
:10126000C16EBE0EC06EC280030EDBCFF0F0050E65
:10127000E15C02E2E16AE552E16EE552E7CFD9FFB7
:101280001200D9CFE6FFE1CFD9FF040EE126010E0F
:10129000F36E030EF3CFDBFF010EE66ED950030FA2
:1012A000E66E000EDA20E66E5FEC0DF0E552E552D8
:1012B000E5520750DF6E010EE66ED950030FE66E61
:1012C000000EDA20E66E5FEC0DF0E552E552E552D5
:1012D000010E07C0DBFFE66ED950030FE66E000E6D
:1012E000DA20E66EECDBE552E552E552020E07C06D
:1012F000DBFF0001E15101E019D0030EDB50EA6A87
:10130000610FE96E000EEA22EF500D0805E0E15191
:1013100003E1230EE16F0AD0E15108E1DF50896E4D
:10132000010EDB508A6E020EDB508B6E040EE15C08
:1013300002E2E16AE552E16EE552E7CFD9FF120021
:101340000201D25126E18250E66EE66A8150E66ED5
:10135000E66A8050E66EE66A610E146E3B0E156E0C
:10136000166A14C0E6FF15C0E6FF16C0E6FFA10E20
:10137000E66E000EE66E28EC1CF0176E0B0EE15EBA
:101380001750A10EE66E000EE66E97EC16F0E552D1
:10139000E55212000201D25108E1E80EE66E3B0E62
:1013A000E66ED5EC16F0E552E5521200D9CFE6FF15
:1013B000E1CFD9FF020EE126DF6A010EDB6A0201EE
:1013C000D25101E07BD0DFCFE9FFEA6AE9BEEA68EB
:1013D000A10EE926000EEA22410EEF6EDF2A010E71
:1013E000DB6A0001F051F36E010EDBCFF4FFF35026
:1013F000F45C3AE2010EDBCFE9FFEA6AE9BEEA6893
:10140000060EEA02F3CFEAFFE902F3CFE9FFF45058
:10141000EA26800EE926020EEA22EECFE6FFEFCFA3
:10142000E6FF5B0E146E3B0E156E166A14C0E6FFE7
:1014300015C0E6FF16C0E6FFDFCF17F0186A17BE2B
:101440001868A10E1726000E182217C0E6FF18C054
:10145000E6FF28EC1CF0196E070EE15E1950050E30
:10146000DF26010EDB2ABDD7DFCFE9FFEA6AE9BE3E
:10147000EA68A10EE926000EEA220A0EEF6EDF2AC4
:10148000DFCFE9FFEA6AE9BEEA68A10EE926000EAD
:10149000EA220D0EEF6EDF2ADFCFE9FFEA6AE9BE2E
:1014A000EA68A10EE926000EEA22EF6AA10EE66EB6
:1014B000000EE66E97EC16F0E552E552020EE15C86
:1014C00002E2E16AE552E16EE552E7CFD9FF120090
:1014D000D9CFE6FFE1CFD9FF040EE126020EF36E6D
:1014E000030EF3CFDBFFE66ED950030FE66E000E5E
:1014F000DA20E66EE4DAE552E552E55207C0DEFF97
:1015000008C0DDFF010EE66ED950030FE66E000E37
:10151000DA20E66ED4DAE552E552E552020E07C053
:10152000DBFF0001E15101E01FD0030EDB50EA6A4E
:10153000610FE96E000EEA22EF500D0805E0E1515F
:1015400003E1230EE16F10D0DECF14F0DDCF15F0F4
:10155000000E145C100E155807E2DECFE9FFDDCF58
:10156000EAFF020EDBCFEFFF040EE15C02E2E16A6C
:10157000E552E16EE552E7CFD9FF1200D9CFE6FF81
:10158000E1CFD9FF040EE126020EF36E030EF3CF76
:10159000DBFFE66ED950030FE66E000EDA20E66E32
:1015A0008EDAE552E552E55207C0DEFF08C0DDFFE6
:1015B0000001E15101E043D0030EDB50EA6A610F04
:1015C000E96E000EEA22EF500D0805E0E15103E15B
:1015D000230EE16F34D0DECF14F0DDCF15F0000E16
:1015E000145C100E155807E2DECFE9FFDDCFEAFFED
:1015F000020EEFCFDBFF0201D25121E1020EDBCF61
:10160000E6FFE66A510E146E3B0E156E166A14C0A4
:10161000E6FF15C0E6FF16C0E6FFA10EE66E000E5F
:10162000E66E28EC1CF0176E070EE15E1750A10E57
:10163000E66E000EE66E97EC16F0E552E552040EEB
:10164000E15C02E2E16AE552E16EE552E7CFD9FFE3
:101650001200D9CFE6FFE1CFD9FF040EE126020E3A
:10166000F36E030EF3CFDBFF040EE66ED950030FCB
:10167000E66E000EDA20E66E22DAE552E552E55219
:101680000750DF6E010EE66ED950030FE66E000EB6
:10169000DA20E66E14DAE552E552E552010E07C093
:1016A000DBFFE66ED950030FE66E000EDA20E66E21
:1016B00006DAE552E552E552020E07C0DBFF0001F3
:1016C000E15101E07DD0030EDB50EA6A610FE96E63
:1016D000000EEA22EF500D0805E0E15103E1230E70
:1016E000E16F6ED0020EDB50010803E22A0EE16FBB
:1016F00067D0010EDB50070803E22A0EE16F60D0CD
:10170000410E146EDF50145C1AE1020EDB500CE146
:10171000010EF36EDB5004E0D890F336E806FCE1EE
:10172000F350E81C92160AD0010EF36EDB5004E071
:10173000D890F336E806FCE1F350921241D0420E05
:10174000146EDF50145C1AE1020EDB500CE1010E46
:10175000F36EDB5004E0D890F336E806FCE1F3507A
:10176000E81C93160AD0010EF36EDB5004E0D8900B
:10177000F336E806FCE1F350931222D0430E146EC8
:10178000DF50145C1AE1020EDB500CE1010EF36E27
:10179000DB5004E0D890F336E806FCE1F350E81C97
:1017A00094160AD0010EF36EDB5004E0D890F336A5
:1017B000E806FCE1F350941203D02A0EE16F00D04A
:1017C000040EE15C02E2E16AE552E16EE552E7CF28
:1017D000D9FF1200D9CFE6FFE1CFD9FF040EE126F1
:1017E000020EF36EF3CFDBFF030EDB6A040EE66E30
:1017F000D950020FE66E000EDA20E66E60D9E5528F
:10180000E552E5520750DF6E010EE66ED950020F29
:10181000E66E000EDA20E66E52D9E552E552E55248
:10182000010E07C0DBFF0001E15101E079D0020E9B
:10183000DB50EA6A610FE96E000EEA22EF500D08F4
:1018400005E0E15103E1230EE16F6AD0010EDB50A8
:10185000070803E22A0EE16F63D0410E146EDF50D9
:10186000145C0FE1010EF36EDB5004E0D890F33608
:10187000E806FCE1F3508014E76E030EE7CFDBFFD0
:101880002BD0420E146EDF50145C0FE1010EF36E8C
:10189000DB5004E0D890F336E806FCE1F350811405
:1018A000E76E030EE7CFDBFF17D0430E146EDF5059
:1018B000145C0FE1010EF36EDB5004E0D890F336B8
:1018C000E806FCE1F3508214E76E030EE7CFDBFF7E
:1018D00003D02A0EE16F24D00201D25121E1030E80
:1018E000DBCFE6FFE66A480E146E3B0E156E166AF5
:1018F00014C0E6FF15C0E6FF16C0E6FFA10EE66EB7
:10190000000EE66E28EC1CF0176E070EE15E175015
:10191000A10EE66E000EE66E97EC16F0E552E5526B
:10192000040EE15C02E2E16AE552E16EE552E7CFC6
:10193000D9FF1200D9CFE6FFE1CFD9FF040EE1268F
:10194000020EF36E030EF3CFDBFF040EE66ED950EA
:10195000030FE66E000EDA20E66EB1D8E552E552CE
:10196000E5520750DF6E010EE66ED950030FE66EAA
:10197000000EDA20E66EA3D8E552E552E552010EDC
:1019800007C0DBFFE66ED950030FE66E000EDA20CB
:10199000E66E95D8E552E552E552020E07C0DBFF30
:1019A0000001E15101E07DD0030EDB50EA6A610FD6
:1019B000E96E000EEA22EF500D0805E0E15103E167
:1019C000230EE16F6ED0020EDB50010803E22A0EF7
:1019D000E16F67D0010EDB50070803E22A0EE16FCA
:1019E00060D0410E146EDF50145C1AE1020EDB5021
:1019F0000CE1010EF36EDB5004E0D890F336E806FC
:101A0000FCE1F350E81C89160AD0010EF36EDB509E
:101A100004E0D890F336E806FCE1F350891241D097
:101A2000420E146EDF50145C1AE1020EDB500CE122
:101A3000010EF36EDB5004E0D890F336E806FCE1CB
:101A4000F350E81C8A160AD0010EF36EDB5004E056
:101A5000D890F336E806FCE1F3508A1222D0430E08
:101A6000146EDF50145C1AE1020EDB500CE1010E23
:101A7000F36EDB5004E0D890F336E806FCE1F35057
:101A8000E81C8B160AD0010EF36EDB5004E0D890F0
:101A9000F336E806FCE1F3508B1203D02A0EE16F17
:101AA00000D0040EE15C02E2E16AE552E16EE5522B
:101AB000E7CFD9FF12001200120012001200D9CF96
:101AC000E6FFE1CFD9FF040EE126030EDB6A000139
:101AD000E15104E0076A086A096A66D1FD0EDBCFAE
:101AE000E9FFFE0EDBCFEAFFEF50EA6A610FE96E15
:101AF000000EEA22EF502C0806E05E0EE16F076A46
:101B0000086A096A51D1FD0EDBCFE9FFFE0EDBCF7B
:101B1000EAFFEF2A2D0E146EFD0EDBCFE9FFFE0E5D
:101B2000DBCFEAFFEF50EA6A610FE96E000EEA22AE
:101B3000EF50145C22E1040E156EFC0EDB50155CB8
:101B40001CE0FC0EDB0406E0030E146EFC0EDB5002
:101B5000145C07E17C0EE16F076A086A096A24D108
:101B60000CD0010EF36E030EF3CFDBFFFD0EDBCFC7
:101B7000E9FFFE0EDBCFEAFFEF2A040E146EFC0E27
:101B8000DB50145C12E0050EE66ED9CFE6FFDACF2B
:101B9000E6FFFD0EDBCFE6FFFE0EDBCFE6FF0ED944
:101BA000146E050EE15E14501FD0FD0EDBCFE9FF71
:101BB000FE0EDBCFEAFFEF50EA6A610FE96E000E1E
:101BC000EA22EFCF14F0156A166A14C0DFFF010E87
:101BD00015C0DBFF020E16C0DBFFFD0EDBCFE9FFF9
:101BE000FE0EDBCFEAFFEF2A030EDB5021E0DFCF52
:101BF00014F0010EDBCF15F0020EDBCF16F00C68EF
:101C00000D680E6814C007F015C008F016C009F082
:101C10004BEC1BF004C014F005C015F006C016F024
:101C200014C0DFFF010E15C0DBFF020E16C0DBFF84
:101C3000FC0EDB5026E1DFCF14F0010EDBCF15F0F8
:101C4000020EDBCF16F01634000E161807E6D88009
:101C50007F0E1454000E1554000E165401E28CD061
:101C6000D9CFE9FFDACFEAFF020ED880EB50FF0AA6
:101C700006E6800EEE5CFF0EEE58FF0EEF5801E216
:101C80007BD0FC0EDB0424E1DFCF17F0010EDBCFAD
:101C900018F0020EDBCF19F01934000E191807E600
:101CA000D880FF0E1754000E1854000E195464E328
:101CB000D9CFE9FFDACFEAFF020ED890EB50000A45
:101CC00006E6000EEE5C000EEE58000EEF5854E3F0
:101CD000020E1A6EFC0EDB501A5C24E1DFCF1BF003
:101CE000010EDBCF1CF0020EDBCF1DF01D34000E09
:101CF0001D1807E6D880FF0E1B547F0E1C54000EE3
:101D00001D543AE3D9CFE9FFDACFEAFF020ED880BB
:101D1000EB50FF0A06E6000EEE5C800EEE58FF0E5A
:101D2000EF582AE3030E1E6EFC0EDB501E5C2DE105
:101D3000DFCF1FF0010EDBCF20F0020EDBCF21F052
:101D40002134000E211807E6D880FF0E1F54FF0E25
:101D50002054000E215410E3D9CFE9FFDACFEAFF77
:101D6000020ED890EB50000A06E6000EEE5C000E64
:101D7000EE58000EEF5809E20001E15106E17E0E37
:101D8000E16F076A086A096A0FD0DFCF14F0010E0D
:101D9000DBCF15F0020EDBCF16F014C007F015C034
:101DA00008F016C009F000D0040EE15C02E2E16A1E
:101DB000E552E16EE552E7CFD9FF1200D9CFE6FF39
:101DC000E1CFD9FF020EE126FB0EDBCFE9FFFC0ECF
:101DD000DBCFEAFFEE6AEE6AEE6A010EDB6AFA0E0C
:101DE000DB50F36E010EDBCFF4FFF350F45C58E2EE
:101DF000FD0EDBCFE9FFFE0EDBCFEAFFEF50EA6A14
:101E0000610FE96E000EEA22EFCFDFFF300EDF5CDC
:101E100045E3DF50390842E3FB0EDBCFE9FFFC0E60
:101E2000DBCFEAFFEECF17F0EECF18F0EFCF19F0CF
:101E30000A0E0C6E0D6A0E6A17C007F018C008F083
:101E400019C009F04BEC1BF004C017F005C018F0E6
:101E500006C019F0300EDF5C1A6E1B6A1C6A175040
:101E60001A24146E18501B20156E19501C20166E63
:101E7000FB0EDBCFE9FFFC0EDBCFEAFF14C0EEFF69
:101E800015C0EEFF16C0EEFFFD0EDBCFE9FFFE0E24
:101E9000DBCFEAFFEF2A010EDB2AA1D7000E02D02A
:101EA000010E00D0146E020EE15C02E2E16AE5521E
:101EB000E16E1450E552E7CFD9FF12000001E15165
:101EC00024E10201D25121E10001EA51E66EE66A05
:101ED0003C0E146E3B0E156E166A14C0E6FF15C05C
:101EE000E6FF16C0E6FFA10EE66E000EE66E28ECD9
:101EF0001CF0176E070EE15E1750A10EE66E000E85
:101F0000E66E97EC16F0E552E55212000201F4512C
:101F1000F51104E1500EF46FC30EF56FF407000ED7
:101F2000F55B0001FC5108E0010E146E6D50020BD0
:101F300001E0010E145C02E18B9015D0FC0509E074
:101F4000020EFC5D06E0030EFC5D03E0050EFC5D89
:101F500002E18B8008D0060EFC5D05E10201F45120
:101F6000F51101E18B70120082B403D0010E03D091
:081F700002D0000E00D01200A7
:081F7800F8EC14F0FB0EDBCFC6
:101F8000F3FFDB06F35000090AE046EC15F0FA0E09
:101F9000B1EC15F0F3E1151CF1E1010E01D0000EDA
:101FA00027EF15F0F8EC14F03B0EE12402E3E168B2
:101FB000E652E16E010EDB6A020EDB6AF90EDBCF40
:101FC000F6FFFA0EDBCFF7FFFB0EDBCFF8FF0800C2
:101FD000F550DF6EDF5002E14BEF14F0250EDF5CB1
:101FE00002E03EEF14F0030EDB6A040EDB6A050E1E
:101FF000DB6A060EDB6A070EDB6A60EC14F02D0E5E
:10200000DF5C0CE02B0EDF5C09E0200EDF5C06E0FD
:10201000230EDF5C03E0300EDF5C1AE1DF50300A94
:1020200014E0130A0FE0030A0AE00B0A05E0060AAF
:10203000E4E1030EDB80E1D7030EDB82DED7030E83
:10204000DB84DBD7030EDB86D8D7030EDB88D5D73E
:102050002A0EDF5C1BE15CEC14F0AAEC14F010E03B
:10206000030EDB8008680968130EDBCF0DF0140E39
:10207000DBCF0EF094EC1BF0040E06C0DBFF03D0A8
:10208000130E93EC14F060EC14F00BD0090EDB6A25
:1020900001EC15F003E075EC15F0FAD7090E93EC9E
:1020A00014F0030EDBB0DB982E0EDF5C1BE160EC5E
:1020B00014F02A0EDF5C0BE15CEC14F0AAEC14F0D7
:1020C00003E1130EE5EC14F060EC14F00BD0090EF4
:1020D000DB6A01EC15F003E075EC15F0FAD7090E98
:1020E000E5EC14F0680EDF5C07E160EC14F0680EBC
:1020F000DF5C1DE1030E18D0740EDF5C17E07A0E72
:10210000DF5C14E0480EDF5C06E0540EDF5C03E0A9
:102110005A0EDF5C02E1020E07D06C0EDF5C03E0BA
:102120006A0EDF5C04E1010E38EC15F0C9DBDF500C
:102130006E0A01E17FD31E0A01E192D1200A01E17A
:102140008FD13F0A01E149D11A0A01E146D10D0AB6
:1021500001E143D1200A01E140D13A0A01E13DD138
:10216000200A01E13AD1260A01E135D10D0A01E147
:1021700032D11A0A01E1D9D0200A4AE0300A1FE020
:10218000460A0EE0250A01E083D3D950F90FE96E23
:10219000FF0EDA20EA6E010EEE5E000EEE5AEE5AE7
:1021A00046EC15F0250EE66E95DB03E1151C01E10A
:1021B00069D342EC15F001E26BD3DB2A69D3080E38
:1021C000DB6A040EDB50010806E2040EDB040AECB5
:1021D00015F0DB508BDB080EDB5009E0030EDB5003
:1021E000010B05E172DB01E04DD3080EDB6A64DB15
:1021F000EFCFDFFFBAEC15F003E1151C01E142D38C
:1022000042EC15F001E3DB2A60DB01E141D33AD374
:10221000070EDB5002080FE186EC15F0030E4DECC3
:1022200015F00E0EEECFDBFF0F0EEECFDBFF100E24
:10223000EECFDBFF20D0F70EDBCF17F0F80EDBCFB1
:1022400018F0020E175E000E185AF70E17C0DBFFCB
:10225000F80E18C0DBFF17C0E9FF18C0EAFF3DEC1D
:1022600015F0166A0E0E14C0DBFF0F0E15C0DBFF53
:10227000100E16C0DBFF0E0EDBCFE6FF0F0EDBCF1E
:10228000E6FF100EDBCFE6FF55EC1DF0E552E55200
:10229000E552130E07C0DBFF140E08C0DBFF060E6D
:1022A000DB5005E0130E81EC15F001E26ADBA5ECD2
:1022B00015F002E2130E37DB68EC15F006E0040EB1
:1022C00081EC15F002E2050E2EDB030EDBB005D02B
:1022D000FCDA01E0D7D2080EDB6A090EDB6A0E0ECB
:1022E000DBCFF6FF0F0EDBCFF7FF100EDBCFF8FFD3
:1022F0000800F550DF6EDF5014E0ABEC15F011E292
:10230000BAEC15F003E1151C01E1BCD2BBDB01E323
:10231000DB2A090EDB2AD9500E0FE96E000ECBDB4B
:10232000E7D7D3DA01E1B4D2ADD2C6DA110EEECFDF
:10233000DBFF120EEDCFDBFF110EDBCFE6FF120E3F
:10234000DBCFE6FF47EC1DF0E552E552130EF3CF6D
:10235000DBFF140EF4CFDBFF060EDB5004E0130EA0
:10236000D0DB01E20EDBA5EC15F002E2130EDBDAA6
:10237000AFDB05E0040EC5DB02E2050ED4DA030E86
:10238000DBB005D0A2DA01E07DD2080EDB6A090ECF
:10239000DB6A110EDBCFE9FF120EDBCFEAFFEFCFD6
:1023A000DFFFDF5014E0D7DB12E2E4DB03E1151CB2
:1023B00001E168D267DB01E3DB2A090EDB2A110E9B
:1023C000DB2ADBCFE9FF120EE8E3DB2AE6D77DDA72
:1023D00001E15ED257D2030EDB8E070EDB0410E163
:1023E00095DB040E5ADB0A0EEECFDBFF0B0EEECFB1
:1023F000DBFF0C0EEECFDBFF0D0EEECFDBFF6CD064
:10240000070EDB5003082CE1030EDBAE0DD0B2DA71
:10241000020E76DAEFCF14F0156A166A176A14AE58
:1024200039D01568166835D0F70EDBCF15F0F80EE9
:10243000DBCF16F0020E155E000E165AF70E15C011
:10244000DBFFF80E16C0DBFF15C0E9FF16C0EAFF80
:10245000EFCF14F00A0E14C0DBFF0B0EDB6A38D08E
:10246000070EDB50020809E1030EDBAE04D059DB96
:1024700016AE10D00ED055DB0DD0030EDBAE12D051
:1024800079DA020E3DDAF9DA166A176A15AE02D069
:1024900016681768E2DA0C0E16C0DBFF0D0E17C0C7
:1024A000DBFF1AD0F70EDBCF16F0F80EDBCF17F0FC
:1024B000020E165E000E175AF70E16C0DBFFF80E5E
:1024C00017C0DBFF16C0E9FF17C0EAFFD6DAC5DA8E
:1024D0000C0EDB6A0D0EDB6A060EDB5005E1010E09
:1024E000F36E050EF3CFDBFF150EDB6A160EDB6A0B
:1024F000D950370F146E000EDA20156E390E14C045
:10250000DBFF3A0E15C0DBFF380EDB6A080EDB6A14
:102510000A0EAEDADF50780A12E0200A10E0280A2C
:102520000CE0200A0AE03F0A06E00D0A02E0200A59
:1025300008E1020E05D0080E03D0080EDF26100EAB
:1025400097DA030EDBBE02D0DB92DB94DB50800B0C
:1025500024E08ADAD890030EEB50000A08E6000E59
:10256000EE5C000EEE58000EEE58000EEE5815E22E
:1025700013DA0B680C680D680E680FEC1DF00A0E7C
:1025800002C0DBFF0B0E03C0DBFF0C0E04C0DBFF41
:102590000D0E05C0DBFF2D0E08D0030EDBA202D00E
:1025A0002B0E03D0DBA408D0200EF36E170EF3CF52
:1025B000DBFF150EDB2A02D0170EDB6A050EDB509F
:1025C00003E1B7D901E189D01A0E146E3C0E156EE5
:1025D000000E166E070EDBCF17F0186A196A1A6A1A
:1025E00017C00BF018C00CF019C00DF01AC00EF097
:1025F000D3D97AEC1DF014500224F36E1550032049
:10260000F46E16500420F86EF4CFF7FFF3CFF6FF08
:102610000800090EF5CFDBFF580EDF5C0FE1610EFD
:10262000F36E090E7BD90AE3200E146E090EDBCF80
:10263000E7FF1450E75E090EE7CFDBFF070EDBCFA5
:1026400014F0156A166A176A0FDA14C00BF015C079
:102650000CF016C00DF017C00EF0EECF06F0EECF66
:1026600007F0EECF08F0EFCF09F07AEC1DF009C0CB
:10267000EDFF08C0EDFF07C0EDFF06C0EFFF390E0C
:10268000DBCFE9FFDB063A0EDBCFEAFF01E2DB0638
:10269000090EDBCFEFFF150EDB2A4BD995E1030EB8
:1026A000DBA61DD06F0EDF5C06E1C1D918E3150E65
:1026B000DB285BDA14D0780EDF5C09E0580EDF5CB3
:1026C00006E0620EDF5C03E0420EDF5C08E1020E12
:1026D000F36E160EF3CFDBFF02D0150EDB6A030E8E
:1026E000DB50100B0EE0040EDBCF14F0050EDB50B8
:1026F000D880145406E2060EDB5003E1040EDB50D2
:1027000034DA95D90AE2050EDBCFE7FF150EDB5070
:10271000E75E050EE7CFDBFF02D0050EDB6A040E95
:10272000DBCF14F0160E45D9D880145414E2160EDF
:10273000DBCFE6FF150EDBCFE6FF040EDBCFE6FFB7
:10274000050EDB50E552E75CE552D880E754E552D0
:10275000D880E7545FD9030EDB50010B0BE1080E64
:10276000DB5008E0B2D801E08DD0080EDB50BED8B7
:10277000080EDB6A170EDB5007E088D9170EF1D977
:1027800003E1151C01E17ED0160EDB5016E07ED968
:10279000300EE66E9FD802E1151C74E077D9DFCFCA
:1027A000E6FFCDEC1CF0E552E552E552F4CF15F012
:1027B0000001F31C02E1151C65E0050EDBCF14F0EF
:1027C000160EDB50D880145409E2050EDBCFE7FF6C
:1027D000160EDB50E75E050EE7CFDBFF300EE66E30
:1027E000050ECBD94FE1390EDB2ADBCFE9FF3A0EDC
:1027F00001E3DB2ADBCFEAFF090EEFCFDBFFDB5083
:102800000EE044D9090EADD902E1151C3BE0390EAA
:10281000DB2ADBCFE9FF3A0EEDE3DB2AEBD755D815
:1028200031E1160EDBCFE6FF080EC3D8E552E724F0
:102830005DD82ED0070EDB50030A1CE0010A14E01D
:10284000030A07E07BD9DBCFEEFF020EDBCFEDFF03
:102850001FD0F5D8196A17AE02D0186819682CD89D
:10286000BCD819C0EEFF14D0EAD817BE186824D817
:10287000B4D80ED063D9DBCFEFFF0AD07BD905E106
:10288000151C03E1F368F46810D0FCD801E3DB2ADF
:1028900079D9E7EF0FF0010EDBCF14F0020EDBCF9A
:1028A00015F014C0F3FF15C0F4FF3B0EE15C02E22B
:1028B000E16AE552E16ECBD029D9020E4DEF15F059
:1028C00061D90800F550DF6E1200200EE66E080E8A
:1028D000BDEF15F0CDEC1CF0E552E552E552F3CF1B
:1028E00014F0F4CF15F00001F31C1200146E156AF9
:1028F000D950010F4DD91450EE261550ED2212007B
:10290000185E000E195AF70E18C0DBFFF80E19C03A
:10291000DBFF18C0E9FF19C0EAFF1200DBCFF4FFAC
:10292000F350F45C1200DB50E76E040EE7CFDBFFE0
:1029300012000A0EDBCF14F00B0EDBCF15F00C0EDD
:10294000DBCF16F00D0EDBCF17F01450151016105C
:1029500017101200130EEECFDBFF140EEDCFDBFFCE
:10296000130EDBCF14F0140EDBCF15F00001800E38
:1029700015141200F70EDBCF18F0F80EDBCF19F0AC
:102980001200050EDB50E66ED950130F01D9E55247
:10299000E750EE6EED6A12000A0EDBCF06F00B0E6A
:1029A000DBCF07F00C0EDBCF08F00D0EDBCF09F00C
:1029B0001200DBCFE6FF150EDBCFE6FF050EDB5086
:1029C000E552E724E552E7241200DB50CED8010E91
:1029D000F36E060EF3CFDBFF1200EE50EFCFEAFFEF
:1029E000E96E16C0EEFF17C0EEFF18C0EEFF120032
:1029F000D9CFE6FFDACFE6FFE1CFD9FFE2CFDAFFAA
:102A00001200DFCFE6FFE66AD4EC1DF0E552E55296
:102A1000F3501200E76E080EE7CFDBFF1200EECF97
:102A200014F0EECF15F0EFCF16F0176A1200050E76
:102A3000DBCF14F0150EDB50D88014541200010EB9
:102A4000DBCF16F0020EDBCF17F0186A1200E5524A
:102A5000E5CFDAFFE7CFD9FF12000A0E14C0DBFF83
:102A60000B0E15C0DBFF1200D9500A0FC8EF15F08E
:102A7000F36E070EF3CFDBFF1200EECF14F0EFCFB3
:102A800015F01200010EDB2A020E1200FC0EDBCF45
:102A9000E6FFFD0EDBCFE6FF1200145E000E155AB6
:102AA000F70E14C0DBFFF80E15C0DBFF14C0E9FF02
:102AB00015C0EAFF1200DA20EA6EEF2AEECFF6FF29
:102AC000000EEF22EECFF7FFEF22EECFF8FF12005D
:102AD000040EDBCFE6FF130EDB50E552E75C9ADF16
:102AE000DB5004DF060EDB501200090EDB500A0D2E
:102AF000F350DF24D00FE76E090EE7CFDBFF60EF66
:102B000014F0DB50F36E050E8EEF14F0F70EDBCFF2
:102B100014F0F80EDBCF15F01200DFCFE6FF6AEFFE
:102B200014F028DF030EECDE0FEF15F0BCEC0FF015
:102B3000E552E552E552E55200091200BDDEEE50C5
:102B4000EFCFEAFFE96E010E1200130EDB50F36EB9
:102B5000040E8EEF14F0040EDB50F36E090E8EEFB0
:102B600014F0DBCFE6FF6AEF14F0E76E050EE7CF57
:102B7000DBFF12008BDF8DEF15F0DBCFE6FF86DF8A
:102B800096EF15F0D950F90FE96EFF0E5BEF15F0D7
:0A2B9000E96E000EDA20EA6E120072
:062B9A00040120511F0B95
:102BA000010801E05BD02051600BE842E842E842B6
:102BB000E842E842010801E051D0245103E0240535
:102BC00001E04CD02151230A48E0010A40E0030A09
:102BD00030E0010A25E0240A22E0070A1FE0010A8A
:102BE0001CE0030A11E0010A01E038D00201030EE3
:102BF000F76F0201E40EF86F020EF96F0001FD930A
:102C00000201080EFC6F2AD00201030EF76F0201C9
:102C1000E40EFA6F020EFB6F21D020D01FD01ED021
:102C20000201030EF76F0201D90EFA6F020EFB6F5D
:102C300015D00201030EF76F0201D90EF86F020ED4
:102C4000F96F0001FD930201070EFC6F07D002012E
:102C5000030EF76F22C4E0F201D000D0120002018F
:102C6000D96BC20EDA6F010EDB6FDC6BDD6BDE6BD6
:102C7000080EDF6FD26BD16B1A0E726E1E0E736E62
:102C80000401000E166F050E176F400E146F04013D
:102C9000196F080E1A6F050E1B6F880E186F04014E
:102CA000480E1E6F050E1F6F400E1C6F1200D9CF0D
:102CB000E6FFE1CFD9FF0201D16B040118BF30D08C
:102CC000FC0EDBCF14F01951D880145403E2FC0E33
:102CD00019C4DBFF0201D16BFC0EDB50D15D19E2A0
:102CE000D151EA6A080FE96E050EEA22EF50E66E4E
:102CF000D151E76EFD0EDBCFE9FFFE0EDBCFEAFF21
:102D0000E750E926000EEA22E552E750EF6ED12B9C
:102D1000E3D70401400E196F1817187D880E181399
:102D20000201D15100D0E552E7CFD9FF1200D9CF2F
:102D3000E6FFE1CFD9FFE6520201D25101E030D0E7
:102D4000DF6ADF2ADF50146E156A145002E1010EAB
:102D5000151801E10BD0FD0EDBCFE9FFDB2AFE0EDB
:102D6000DBCFEAFF01E3DB2AEF50EBE1DF50146E2B
:102D7000156AD950FD0FE96EFF0EDA20EA6E145085
:102D8000EE5E1550ED5ADF06FD0EDBCFD3F2FE0EE0
:102D9000DBCFD4F2DFCFD7F20201D86B010ED26FB6
:102DA000E552E552E7CFD9FF1200D9CFE6FFE1CFD8
:102DB000D9FFE6520201D25101E031D0DF6ADF2AA9
:102DC000DF50146E156AFF0E141801E1155001E171
:102DD0000CD0FD0EDBCFF6FFDB2AFE0EDBCFF7FFBC
:102DE00001E3DB2A0800F550EAE1DF50146E156AB2
:102DF000D950FD0FE96EFF0EDA20EA6E1450EE5E38
:102E00001550ED5ADF06FD0EDBCFD3F2FE0EDBCF01
:102E1000D4F2DFCFD7F20201010ED86FD26FE552A4
:102E2000E552E7CFD9FF1200D9CFE6FFE1CFD9FFB6
:102E3000E65204011CBF6BD0030E0201D25D01E11A
:102E4000D26BD25101E163D0020ED25D06E10401E2
:102E50001D6B0201030ED26F54D0D20552E1400E19
:102E6000146E156AD751145C000E155803E2400E1B
:102E7000DF6E02D0D7C2DFFFDFCF1DF4DF50D75D9A
:102E8000D76F480ED56F050ED66FD80515E1DF5008
:102E900012E0D3C2F6FFD4C2F7FF0800F550D5C246
:102EA000E9FFD6C2EAFFEF6ED52B000ED623D32B57
:102EB000D423DF06ECD713D0DF5011E0D3C2E9FFF3
:102EC000D4C2EAFFEF50D5C2E9FFD6C2EAFFEF6EE7
:102ED000D52B000ED623D32BD423DF06EDD7D75125
:102EE00010E104011D51146E156A400E141801E121
:102EF000155004E10201020ED26F03D00201030E4D
:102F0000D26F400E04011C171C7D880E1C13E55265
:082F1000E552E7CFD9FF1200E2
:082F180004012051600BE842A6
:102F2000E842E842E842E842000901E055D0215178
:102F3000070A51E00B0A4FE0070A40E0010A2CE0C3
:102F40000B0A28E0020A26E0030A22E0080A12E03F
:102F5000010A0EE00F0A0AE0030A01E03CD0020178
:102F6000010EF76F0001040EFC6F36D036D834D056
:102F700090D832D00201010EF76F0201FE0EF86FF9
:102F8000000EF96F0001FD930201010EFC6F24D0C9
:102F9000A8D822D0F4D820D00201010EF76F040186
:102FA00024510201F86FF96BFF0EF827000EF92388
:102FB0000001FD930201010EFC6F0ED00201010E13
:102FC000F76F04012451EA6AFF0FE96E000EEA224E
:102FD00022C4EFFF01D000D01200800E0401205D5A
:102FE00057E12351030A34E0010A10E0030A01E02B
:102FF0004DD00201010EF76F0201820EF86F370EFD
:10300000F96F120E0201FC6FFD6B40D00201010E40
:10301000F76F04012251F66EF76AD890F636F7364C
:10302000430EF626380EF7220900F5CFF8F20A0013
:10303000F5CFF9F2020E0201F76AF825F66EF951A2
:10304000F7220900F5CFFCF20A00F5CFFDF21ED001
:103050000201010EF76F04012251F66EF76AD89053
:10306000F636F736470EF626380EF7220900F5CF6A
:10307000F8F20A00F5CFF9F2F8C2F6FFF9C2F7FF4D
:103080000800F5500201FC6FFD6B00D00001FD83CC
:1030900012000201010EF76F0F0EE66E710EE66E62
:1030A0000F0EE66E36EC1BF0E552E552E552010ECE
:1030B000E66EFF0EE66E000EE66E36EC1BF0E55295
:1030C000E552E55222C4FEF00401225104E1000160
:1030D000050EFC6F05D00001060EFC6F2FEC16F0FC
:1030E00012000401286B296B040120511F0B020AF6
:1030F00014E0030A0EE0010A01E033D00201010EE0
:10310000F76F040128810001FDA102D0040128838A
:1031100028D00201010EF76F24D00201010EF76FD3
:10312000040124510F0B080DF350156A000F146EA3
:10313000040E15222451800B01E0010E040DF35002
:1031400002011424FA6F000E1520FB6FFAC2E9FF8A
:10315000FBC2EAFFEF50040B03E00401010E286FED
:1031600000D00201F7050AE10201280EF86F040EF3
:10317000F96F0001FD930201020EFC6F12000401C1
:10318000220510E120511F0B00090CE10201010E84
:10319000F76F030E0401215D03E10001FD8102D000
:1031A0000001FD91040122513AE120511F0B020858
:1031B00036E124510F0B000932E00201010EF76FD6
:1031C000040124510F0B080DF350156A000F146E03
:1031D000040E15222451800B01E0010E040DF35062
:1031E00002011424FA6F000E1520FB6F030E040178
:1031F000215D07E1840EFAC2E9FFFBC2EAFFEF6E30
:103200000ED024AF06D0FAC2E9FFFBC2EAFFEF6A94
:1032100006D0880EFAC2E9FFFBC2EAFFEF6E120089
:103220006C5002E0000E01D0010E00090BE0040119
:1032300000513C0BE842E8420D0802E10CD801D0F5
:1032400040D808D06C5002E0000E01D0010E0409F5
:1032500001E047D81200D9CFE6FFE1CFD9FFE6520F
:103260000201F66BF76BFC6BFD6B8CEC17F0DF6A01
:10327000DF50146E156A010E145C000E15581BE227
:103280000201F75101E017D0F76ADF34FE0BF73681
:10329000F66E4D0EF626380EF7220900F5CF14F023
:1032A0000800F5CF15F004D015C0FAFF1450F96EE0
:1032B000FBDFDF2ADDD7DDD8E552E552E7CFD9FFC6
:1032C0001200020E0201F65D0AE196D8040100BD6B
:1032D00003D0C80E006F02D0880E006F01D00FD946
:1032E0001200040E0001FC5D0AE122C46EFF6E5064
:1032F000000803E2050EFC6F02D0030EFC6F020112
:10330000F6050AE10BD8040104BD03D0C80E046F12
:1033100002D0880E046F01D0F2D81200D9CFE6FF98
:10332000E1CFD9FF020EE1260201080EFC5D000E7E
:10333000FD5905E2FCC2DEFFFDC2DDFF03D0080E31
:10334000DE6EDD6A040104930491010EDB50041368
:10335000DFCF05F4000EDB500201FC5F010EDB50F5
:10336000FD5B280EFA6F040EFB6F0001FDA31ED05B
:10337000D9CFE9FFDACFEAFFEE50ED1016E0F8C240
:10338000F6FFF9C2F7FF0800F550FAC2E9FFFBC2E9
:10339000EAFFEF6E0201FA2B000EFB23F82BF92354
:1033A000DF06010E01E2DB06E3D71CD0D9CFE9FF2F
:1033B000DACFEAFFEE50ED1015E0F8C2E9FFF9C2EE
:1033C000EAFFEF50FAC2E9FFFBC2EAFFEF6E02012B
:1033D000FA2B000EFB23F82BF923DF06010E01E286
:1033E000DB06E4D7020EE15C02E2E16AE552E16E3F
:1033F000E552E7CFD9FF1200D9CFE6FFE1CFD9FFE1
:10340000020EE126030E04010015E76E010EE7CF60
:10341000DBFF01C4DFFFDE500201FC27DD50FD238E
:10342000280EF86F040EF96FD9CFE9FFDACFEAFF63
:10343000EE50ED1014E0F8C2E9FFF9C2EAFFEF50D8
:10344000FAC2E9FFFBC2EAFFEF6EFA2B000EFB2384
:10345000F82BF923DF06010E01E2DB06E5D7020EA9
:10346000E15C02E2E16AE552E16EE552E7CFD9FFA5
:1034700012000201F7510CE10401080E016F200E49
:10348000026F040E036F840E006F0401046F35D0C9
:10349000040120AF22D00201FC510401265D02018B
:1034A000FD510401275904E226C4FCF227C4FDF2B1
:1034B00035DF0201010EF66F0401080E016F200EC8
:1034C000026F040E036F800E006F0401280E066F5A
:1034D000040E076FC80E046F10D00201020EF66FC3
:1034E0000401056BC80E046F0401080E016F280E5D
:1034F000026F040E036FC80E006F6D981200020178
:10350000F66B0401080E016F200E026F040E036FAC
:0A351000880E006F0401046B120026
:06351A006DA60FD802D0DF
:103520006DB613D80001FC0508E16DBA06D0686AD3
:10353000696A69806988020EFC6F12006D6A696AA7
:103540006D860001010EFC6F12006D6A696A000150
:10355000FC6B1200A5EF1AF00001FC5101E13AD01A
:103560006850040B04E06950040B01E03CD86DB2D4
:1035700031D06850010B04E06950010B01E054D8D0
:103580006850100B04E06950100B01E024D868501B
:10359000400B04E06950400B01E03BD86850200B21
:1035A00004E06950200B01E036D86850020B04E0BB
:1035B0006950020B01E036D8030E0001FC5D01E208
:1035C00009D06850080B06E06950080B03E010ECC6
:1035D00019F068961200698468986D82A19AA08A91
:1035E0000300A09A12006D92699468941200000181
:1035F000FDA10ED0F8DF6D840201080EFE6F070EEC
:10360000FF6FFE07000EFF5BFE51FF11FAE16D94A4
:103610001200689C120070A003D07FEC1AF070902A
:10362000689A1200689212006A6A686A9F0E6B6E4E
:103630007B0E696E6E6A0F0EE66E710EE66E0F0EF1
:10364000E66E14D8E552E552E552160E706E68A685
:1036500002D06896FCD76D987FEC1AF00001FD91BE
:103660000001FE6B0001030EFC6F1200D9CFE6FFD4
:10367000E1CFD9FFFD0EDBCFE9FFFE0EDBCFEAFF86
:10368000FC0EDB5004E0EE6AFC0EDB06F9D7E552D7
:06369000E7CFD9FF120094
:0A36960009C013F008C012F007C0CD
:1036A00011F007500C02F4CF05F0F3CF04F00850EE
:1036B0000D02F4CF07F0F3CF06F00C02F35005260D
:1036C000F4500622E86A072211500D02F350052635
:1036D000F4500622E86A072209500C02F35006262D
:1036E000F450072209500D02086AE86A0822F350D4
:1036F0000726F450082211500E02F3500626F4500B
:103700000722096AE86A0822092212500E02F350C1
:103710000726F4500822E86A092213500E02F350DB
:103720000826F4500922000C09C013F008C012F05A
:1037300008500D02F4CF07F0F3CF06F009500E0247
:10374000F4CF09F0F3CF08F00D02F3500726F45040
:103750000822E86A092212500E02F3500726F4509C
:103760000822E86A09220EAEBAEF1BF01250085E7A
:103770001350095A13AE000C0D50085E0E50095A32
:02378000000C3B
:0E3782001201000202000008D8040A00000034
:103790000102000109024300020100803209040015
:1037A00000010202010005240010010424020205A8
:1037B0002406000105240100010705820308000218
:1037C00009040100020A000000070503024000008E
:1037D000070583024000000403090434034D006917
:1037E00000630072006F00630068006900700020D1
:1037F0000054006500630068006E006F006C006F8D
:103800000067007900200049006E0063002E00343C
:10381000034300440043002000520053002D0032B7
:103820000033003200200045006D0075006C00611F
:1038300000740069006F006E002000440065006D98
:0F384000006F0094379437D737DB370F389A2B48
:10385000D9CFE6FFDACFE6FFE1CFD9FFE2CFDAFF3B
:10386000E652E652E652E652D950F90F146EFF0EB8
:10387000DA20156E020E14C0DBFF030E15C0DBFF4D
:10388000020EDBCFE6FF030EDBCFE6FFF90EDBCF48
:10389000E6FFFA0EDBCFE6FFFB0EDBCFE6FFD950EB
:1038A000FC0FE66EFF0EDA20E66ED2EC0FF0146E1F
:1038B000070EE15C02E2E16AE552E16E1450F3CFDB
:1038C000DEFFF4CFDDFFFC0EDBCFE9FFFD0EDBCF2B
:1038D000EAFFEF6ADECF14F0DDCF15F014C0F3FF7E
:1038E00015C0F4FF040EE15C02E2E16AE552E16E0C
:0C38F000E552E5CFDAFFE7CFD9FF120068
:0438FC002A0EF66E2C
:10390000080EF76E000EF86E00010900F550F76F13
:103910000900F550F86F03E1F76701D03DD00900C9
:10392000F550F26F0900F550F36F0900F550F46F90
:1039300009000900F550E96E0900F550EA6E09002A
:1039400009000900F550F56F0900F550F66F090000
:103950000900F6CFF9F0F7CFFAF0F8CFFBF0F2C09C
:10396000F6FFF3C0F7FFF4C0F8FF0001F55302E1E2
:10397000F65307E00900F550EE6EF507F8E2F6079A
:10398000F9D7F9C0F6FFFAC0F7FFFBC0F8FF000156
:0A399000F707000EF85BBFD7120026
:06399A00D9CFE6FFDACFF1
:1039A000E6FFE1CFD9FFE2CFDAFFFB0EDBCF14F069
:1039B000FC0EDBCF15F00001800E15141AE1FB0E92
:1039C000DBCFE9FFFC0EDBCFEAFFEECFF3FFEDCF5D
:1039D000F4FFEE2A000EEF22F3CFE9FFF4CFEAFF67
:1039E000FD0EDBCFEFFFEF50156AF36E15C0F4FF4D
:1039F00010D0FB0EDB50FE0806E1FD0EDBCFE6FF2C
:103A0000E6EC1DF005D0FD0EDBCFE6FF16EC1EF058
:0E3A1000E552E552E5CFDAFFE7CFD9FF12000D
:023A1E00065050
:103A20000B02F3CF02F0F4CF03F00C02F3500326A5
:103A3000000EF420046E06500D02F3500426000E12
:103A4000F420056E06500E02F350052607500B02B7
:103A5000F3500326F4500422000E052207500C02F6
:103A6000F3500426F450052207500D02F3500526AA
:103A700008500B02F3500426F450052208500C02A3
:0E3A8000F350052609500B02F35005261200E4
:023A8E00FE0E2A
:103A9000E3CFE9FFFF0EE3CFEAFFF36AF46AEE52E9
:103AA00003E0F34AF42AFBD71200FF0EE3CFF8FF3E
:103AB000E552FF0EE3CFF7FFE552FF0EE3CFF6FF2F
:103AC000E552E66AE66AE66A0900F55209E0FD0E8B
:103AD000E32A05E1FE0EE32A02E1FF0EE32AF4D712
:103AE000FD0EE3CF07F0FE0EE3CF08F0FF0EE3CFAD
:043AF00009F01200C7
:0C3AF400056A046A036A026A200EE76E8D
:103B0000D8900636073608360936023603360436AC
:103B100005360B50025C0C5003580D5004580E50E3
:103B2000055809E30B50025E0C50035A0D50045A1D
:0C3B30000E50055A062AE72EE4D71200BA
:043B3C0053746174E9
:103B400075733D25690A0D0050492C2531750A0D04
:103B5000004D522C253033750A0D002C253034755C
:103B600000492C253033692C253033692C2530331E
:043B7000690A0D00D1
:0C3B740005D810D86CEC05F0FCD712004E
:103B80000F0EC112140E6F6E0001FC6B0001FD6B75
:103B90000001FE6BEAEF04F08DEC1AF06FBE02D06C
:083BA000ACEC1AF014EF17F071
:083BA800F36AF46AFF0EE12448
:103BB000E96EFF0EE220EA6EED6607D02F0EEF648D
:0C3BC00004D03A0EEF6001D0F32A12008E
:043BCC00FF0EE350B5
:103BD000ACBA04D0AF6AAB8EAC8A949CACA2FED7D0
:083BE000AD6EF36EF46A1200F1
:083BE8005542572046572044C6
:103BF0002056657273696F6E20312E322E300A0D99
:013C000000C3
:0E3C020013EE00F023EE00F0F86A019C7EEC59
:0A3C10001CF0BAEC1DF0FDD7120005
:063C1A0030313233343575
:0B3C2000363738396162636465660066
:023C2C00120084
:023C2E00000094
:083C300000004100000000004B
:00000001FF
